:020000020000FC
:1000000039C038C037C003D002D0D89808958CE3E7
:100010009FEFD8980000D89A00009A95D1F78A955A
:10002000B9F708958CE39FEF000000000000000086
:100030000000000000009A95B9F78A95A1F708958D
:100040007A95F2E0ECE8C895872F3496C895402D54
:100050004F3FB1F38A958030C1F7402D440F440FD4
:10006000440F440F3196C895400D3196C895402DE8
:100070000895089582E08EBF8FE58DBF8FEF8ABB14
:1000800080E087BB8FEF84BB80E081BB80991DC07F
:10009000C9DF40E045BB809918C0B09905C0C2DFF8
:1000A000B09BFECFBFDFAFDFB19906C0BBDFB19B16
:1000B000FECFB8DF45E045BBB299EDCFB3DFB29BD1
:1000C000FECFB0DF46E045BBE6CF81991EC0AADF78
:1000D00041E045BB819919C0B09906C0A3DFB09B30
:1000E000FECFA0DF44E045BBB19906C09BDFB19BCA
:1000F000FECF98DF45E045BBB299ECCF93DFB29BD2
:10010000FECF90DF46E045BBE5CF82991EC08ADF77
:1001100042E045BB829919C0B09906C083DFB09B0D
:10012000FECF80DF44E045BBB19906C07BDFB19BC9
:10013000FECF78DF45E045BBB299ECCF73DFB29BD1
:10014000FECF70DF46E045BBE5CF83991EC06ADF76
:1001500043E045BB839919C0B09906C063DFB09BEB
:10016000FECF60DF44E045BBB19906C05BDFB19BC9
:10017000FECF58DF45E045BBB299ECCF53DFB29BD1
:10018000FECF50DF46E045BBE5CF84991EC04ADF75
:1001900044E045BB849919C0B09906C043DFB09BC9
:1001A000FECF40DF44E045BBB19906C03BDFB19BC9
:1001B000FECF38DF45E045BBB299ECCF33DFB29BD1
:1001C000FECF30DF46E045BBE5CF85991EC02ADF74
:1001D00045E045BB859919C0B09906C023DFB09BA7
:1001E000FECF20DF44E045BBB19906C01BDFB19BC9
:1001F000FECF18DF45E045BBB299ECCF13DFB29BD1
:10020000FECF10DF46E045BBE5CF86991EC00ADF72
:1002100046E045BB869919C0B09906C003DFB09B84
:10022000FECF00DF44E045BBB19906C0FBDEB19BC9
:10023000FECFF8DE45E045BBB299ECCFF3DEB29BD2
:10024000FECFF0DE46E045BBE5CF87991EC0EADE73
:1002500047E045BB879919C0B09906C0E3DEB09B63
:10026000FECFE0DE44E045BBB19906C0DBDEB19BCA
:10027000FECFD8DE45E045BBB299ECCFD3DEB29BD2
:10028000FECFD0DE46E045BBE5CF00CF0000002129
:1002900000010021000201210003022100040321CA
:1002A000000504210006052100000021FFFFFFFFDB
:00000001FF
